:020000040000FA
:04000000CB303A289F
:040004000034003490
:08000800A000030EA100831209
:100010008B1C32288B1032181428B21C3228643002
:10002000010203183128182800001628172818285C
:1000300019281A281B281C281D281E281F283210A2
:10004000B214A810031005190314AA0DA90DA80DC8
:10005000B10B322832152A08AF002908AE00280853
:10006000AD00B21081010B11210E8300A00E200EF5
:02007000090085
:0C007400203084008001840A80300402E7
:10008000031C3C281230B100E22183160C30850598
:1000900087018312850187010730990000309A009B
:1000A000103083168E008312603083168F00831207
:1000B0000030831691009F008312C83083168100A0
:1000C000831231309000003083168C008312103080
:1000D0008B00BD1B7128851971286400851D6D2852
:1000E000F522DC2281018E018F010B118B100B1088
:1000F0008C018B17892032199F20B40B872803109D
:1001000085190314BA0DF0303A02031945211B2357
:100110007A286400321808000B1D08000B11B21079
:1001200032141230B100051D9A28331483160113BE
:10013000831208003310831601178312080032114E
:100140000130B7008B132030370783169B001C1437
:100150001A088312A400A500C030A5061030370786
:1001600083169B001C141A088312A3000030370763
:1001700083169B001C141A088312A2008B17331CD1
:10018000C72822090339A200A309A409A509220846
:100190002D02031D3F2923082E02031D3F29240899
:1001A0002F02031D3F2901303702031DDC283E18B2
:1001B000DC283E143F14042202303702031DE528D8
:1001C000BE18E528BE143F14102203303702031D69
:1001D000EE283E19EE283E153F141C22043037024B
:1001E000031DF728BE19F728BE153F142822053035
:1001F0003702031D00293E1A00293E163F143422FF
:1002000006303702031D0929BE1A0929BE163F14FC
:10021000432207303702031D12293E1B12293E17C5
:100220003F14552208303702031D1B29BE1B1B2912
:10023000BE173F14602209303702031D24295E18BF
:1002400024295E143F146B220A303702031D2D2926
:10025000DE182D29DE143F1476220B303702031DE1
:1002600036295E1936295E153F1481220C3037027B
:10027000031D3F29DE193F29DE153F148F22B70ADF
:100280000D30370203180800A2280130B600B40070
:10029000B500B70085018701B2138920B40B5D2931
:1002A000031085190314BA0DF0303A02031984299A
:1002B000B50B5D299630B5008E21321D4D293211C6
:1002C000331C67292D090339AD00AE09AF092F1C76
:1002D000B2132F1C4D29B21B4D292E184D29B217D0
:1002E0008B1320303707BC002F08BB00CD21103006
:1002F0003707BC002E08BB00CD2100303707BC00FB
:100300002D08BB00CD218B1785018701B70AB601E7
:100310000D303702031C4D29DC2208000130370262
:100320000319A022023037020319A5220330370235
:100330000319AA22043037020319AF22053037020D
:100340000319B422063037020319B92207303702E5
:100350000319BE22083037020319C32209303702BD
:100360000319C8220A3037020319CD220B30370295
:100370000319D2220C3037020319D72208003F1C80
:1003800008003F101030BC003E08BB00CD213030CB
:10039000BC005E08BB00CD2108008B133B08831610
:1003A0001C159A0083123C0883169B0055309D0053
:1003B000AA309D009C1464009C18DB291C11831238
:1003C0008B170800831600309B001C141A08831238
:1003D000BD00831610309B001C141A088312BE0047
:1003E000831630309B001C141A088312DE00FF3085
:1003F000C800CA15CB15CC15CD15CE15CF15D01507
:10040000D115D215D3150800C130BE05FF30DE0569
:100410000130C405C0000030C200C6005F100800F3
:10042000C230BE05FF30DE050230C405C00000301A
:10043000C200C6005F100800C430BE05FF30DE05F4
:100440000630C405C0000030C200C6005F100800BE
:10045000C830BE05FF30DE050A30C405C0000030DC
:10046000C200C6005F100800D030BE05FF30DE05B8
:100470003D181030BD181130C405C0000030C20056
:10048000C6005F100800E030BE05FF30DE053D18F5
:100490001830BD181930C405C0001830C200C6009D
:1004A0005F105F17C411441208007F30BE05C030D2
:1004B000DE050830C505C1000030C300C7000800D4
:1004C000BF30BE05C030DE051030C505C1000030AC
:1004D000C300C70008003F30BE05C130DE05303024
:1004E000C505C1000030C300C70008003F30BE058D
:1004F000C230DE055030C505C1000030C300C70062
:1005000008003F30BE05C430DE053D188030BD1800
:100510008830C505C1000030C300C70008003F3067
:10052000BE05C830DE053D18C030BD18C830C50551
:10053000C100C030C300C700DF174513C513080052
:100540001030850600308706080020308506003010
:100550008706080021308506003087060800223013
:1005600085060030870608000030850602308706C1
:100570000800023085060230870608000030850634
:100580000430870608000030850601308706080021
:1005900000308506213087060800003085061130BE
:1005A00087060800003085060830870608000030FE
:1005B00085061830870608003E180422BE1810224F
:1005C0003E191C22BE1928223E1A3422BE1A43228A
:1005D0003E1B5522BE1B60225E186B22DE1876225F
:1005E0005E198122DE198F220800B601B401B5011F
:1005F0003D1CFD2ABD01BD14FF2ABD013D143D086F
:10060000B6006400032B042B052B062B072BFF30B1
:10061000B51B8500B51F8501B40B012BB50B012B54
:100620000310B60CB608031D012B0030BC003D08BA
:10063000BB00CD2108008F08031908008F01783016
:100640008E00C80F452DC80A441C4B2B461C3C2B62
:10065000CA1C2D2BCA014A15592B4A1D322BCA011F
:10066000CA15592BCA1D372BCA014A16592B4A1EC7
:10067000592BCA01CA14592B4A1D412BCA014A16CB
:10068000592BCA1D462BCA014A16592B4A1E592BF3
:10069000CA01CA14592BCA1C502BCA014A15592B1E
:1006A0004A1D552BCA01CA15592B4A1E592BCA017E
:1006B0004A15C41C802BC61C712BCB1C622BCB0192
:1006C0004B158E2B4B1D672BCB01CB158E2BCB1DCA
:1006D0006C2BCB014B168E2B4B1E8E2BCB01CB14D0
:1006E0008E2B4B1D762BCB014B168E2BCB1D7B2BD4
:1006F000CB014B168E2B4B1E8E2BCB01CB148E2B8E
:10070000CB1C852BCB014B158E2B4B1D8A2BCB0184
:10071000CB158E2B4B1E8E2BCB014B15441DB52BB1
:10072000461DA62BCC1C972BCC014C15C32B4C1D66
:100730009C2BCC01CC15C32BCC1DA12BCC014C1672
:10074000C32B4C1EC32BCC01CC14C32B4C1DAB2B89
:10075000CC014C16C32BCC1DB02BCC014C16C32B9B
:100760004C1EC32BCC01CC14C32BCC1CBA2BCC01FC
:100770004C15C32B4C1DBF2BCC01CC15C32B4C1ED1
:10078000C32BCC014C15C41DEB2BC61DDC2BCD1C83
:10079000CD2BCD014D155F13F92B4D1DD22BCD0166
:1007A000CD15F92BCD1DD72BCD014D16F92B4D1E97
:1007B000F92BCD01CD14F92B4D1DE12BCD014D169B
:1007C000F92BCD1DE62BCD014D16F92B4D1EF92B26
:1007D000CD01CD14F92BCD1CF02BCD014D15F92BEE
:1007E0004D1DF52BCD01CD15F92B4D1EF92BCD014E
:1007F0004D155F1B222C441E222C461E132CCE1C92
:10080000042CCE014E15302C4E1D092CCE01CE15D8
:10081000302CCE1D0E2CCE014E16302C4E1E302C00
:10082000CE01CE14302C4E1D182CCE014E16302C7D
:10083000CE1D1D2CCE014E16302C4E1E302CCE015E
:10084000CE14302CCE1C272CCE014E15302C4E1D34
:100850002C2CCE01CE15302C4E1E302CCE014E1538
:10086000C51D572CC71D482CCF1C392CCF014F1547
:10087000652C4F1D3E2CCF01CF15652CCF1D432C71
:10088000CF014F16652C4F1E652CCF01CF14652C60
:100890004F1D4D2CCF014F16652CCF1D522CCF0173
:1008A0004F16652C4F1E652CCF01CF14652CCF1C25
:1008B0005C2CCF014F15652C4F1D612CCF01CF153E
:1008C000652C4F1E652CCF014F15451E8C2C471EE5
:1008D0007D2CD01C6E2CD00150159A2C501D732CE1
:1008E000D001D0159A2CD01D782CD00150169A2CFE
:1008F000501E9A2CD001D0149A2C501D822CD0015D
:1009000050169A2CD01D872CD00150169A2C501EB0
:100910009A2CD001D0149A2CD01C912CD0015015B7
:100920009A2C501D962CD001D0159A2C501E9A2C22
:10093000D0015015C51EC12CC71EB22CD11CA32C32
:10094000D1015115CF2C511DA82CD101D115CF2C7F
:10095000D11DAD2CD1015116CF2C511ECF2CD10160
:10096000D114CF2C511DB72CD1015116CF2CD11D34
:10097000BC2CD1015116CF2C511ECF2CD101D1143A
:10098000CF2CD11CC62CD1015115CF2C511DCB2CF5
:10099000D101D115CF2C511ECF2CD1015115451F9E
:1009A000F72C471FE82CD21CD92CD2015215DF138B
:1009B000052D521DDE2CD201D215052DD21DE32CA2
:1009C000D2015216052D521E052DD201D214052D2D
:1009D000521DED2CD2015216052DD21DF22CD20142
:1009E0005216052D521E052DD201D214052DD21CF2
:1009F000FC2CD2015215052D521D012DD201D2150C
:100A0000052D521E052DD2015215DF1B2E2DC51F9F
:100A10002E2DC71F1F2DD31C102DD30153153C2D78
:100A2000531D152DD301D3153C2DD31D1A2DD301E4
:100A300053163C2D531E3C2DD301D3143C2D531D76
:100A4000242DD30153163C2DD31D292DD30153162C
:100A50003C2D531E3C2DD301D3143C2DD31C332DE0
:100A6000D30153153C2D531D382DD301D3153C2DE7
:100A7000531E3C2DD3015315BF214008C40041082B
:100A8000C5005F18DF145F1CDF104808C9000C3078
:100A90004A05031D05120C304B05031D85120C3051
:100AA0004C05031D05100C304D05031D85100C3041
:100AB0004E05031D87100C304F05031D07110C3028
:100AC0005005031D07100C305105031D87120C3013
:100AD0005205031D07120C305305031D87114908E9
:100AE0000E0203189F2D12304A05031D0516123001
:100AF0004B05031D851612304C05031D05141230DD
:100B00004D05031D851412304E05031D8714123048
:100B10004F05031D071512305005031D0714123031
:100B20005105031D871612305205031D071612309A
:100B30005305031D8715FF304802031908008F086D
:100B4000031D0800892049080E02031C9F2D183040
:100B50004A05031D051206304A05031D0516183007
:100B60004B05031D851206304B05031D85161830F5
:100B70004C05031D051006304C05031D05141830E7
:100B80004D05031D851006304D05031D85141830D5
:100B90004E05031D871006304E05031D87141830BF
:100BA0004F05031D071106304F05031D07151830AB
:100BB0005005031D071006305005031D071418309B
:100BC0005105031D871206305105031D8716183085
:100BD0005205031D071206305205031D0716183073
:100BE0005305031D871106305305031D87150800A3
:084000000300030006000900A3
:02400E00CC33B1
:10420000010003000300030003000200020002009B
:104210000200000000000000000003000300030093
:10422000020000000000000000000000000000008C
:104230000000C000C000C000C000C000C000C0003E
:10424000FF00C300F300CF00FF00C300F300CF0066
:10425000FF00C300F300CF00FF00C300F300CF0056
:104260000100FF00FF00FF00FF00FF00FF00FF0054
:10427000FF00FF00FF00FF00FF00FF00FF00FF0046
:10428000FF000300FF00FF00FF00FF00FF00FF0032
:10429000FF00FF00FF00FF00FF00FF00FF00FF0026
:1042A000FF00C000FF00FF00FF00FF00FF00FF0055
:1042B000FF00FF00FF00FF00FF00FF00FF00FF0006
:1042C000FF00FF00FF00FF00FF00FF00FF00FF00F6
:1042D000FF00FF00FF00FF00FF00FF00FF00FF00E6
:1042E000FF00FF00FF00FF00FF00FF00FF00FF00D6
:1042F000FF00FF00FF00FF00FF00FF00FF00AA001B
:00000001FF
